:1000000009C018951895189518951895189518956C
:10001000189518958FE98DBFC8E8E4E84E2EDD27C6
:100020005D2EEEE3F0E0A0E6B0E0A89584B7082EE0
:10003000877F84BF88E1992781BD91BD88278D93F3
:100040003197E9F7662486E886B980E087B9B898E1
:10005000BB98BC9ABA9AB99A80E080936800809164
:1000600069008F7780936900AAE685D180E080934C
:100070006200B9988CE291E066D1B19B16C0B99A42
:10008000C19AE3E0F0E050D1C198B6D0A3E60D915B
:100090001C9141E050E0040F151FA6E60D931C9340
:1000A000E0E0F0E0A6E67BE775D1B99AB09972C0BE
:1000B000A9E68C9187FB0EF426C081E08093650051
:1000C000009165000F3010F009F017C084EF91E047
:1000D0003AD1B09B02C0C298E9CFC19888EC90E0B9
:1000E00032D1C19A88EC90E02ED1C198C29AA5E68F
:1000F0008C918F5F8C9308F4E3CF809169008068C6
:1001000080936900C298C198B998B19B01C0E8C0BA
:10011000B99AC19A84EF91E016D1C49AE1E0F0E077
:1001200003D1C19A69D0E0E0F0E0A6E644D1A6E6AA
:100130004D915C91A3E60D911C910417150710F0E9
:1001400009F001C004C080E08093620015C0C1982E
:1001500080E590E0F8D0C19AA2E68C918F5F8C93F5
:1001600084E690E0F0D0009162000A3009F004C00B
:1001700080E08093620071C0AAE6CFD0AAE60D911C
:100180001C910C3251E0150709F003C0AAE6F3D028
:100190008AC02FC0AAE6EFD0C498A9E68C9187FB4D
:1001A0000EF01EC081E080936500009165000A306A
:1001B00010F009F00FC0C29AC19888EC90E0C3D04B
:1001C000C19A88EC90E0BFD0A5E68C918F5F8C93AC
:1001D00008F4EBCF809169008F7780936900C29813
:1001E000C198E1E0F0E0A0D0C19AE1E0F0E09CD05D
:1001F000C1985CCFF894FFCFA3E6BDD0379A81E0D9
:1002000080936500009165000A3010F009F023C06A
:1002100007B10C7F036007B9A5D0A0E68D939C932E
:10022000A3E64D915C91A0E60D911C910417150772
:1002300010F009F001C006C0A0E68D919C91A3E6E4
:100240008D939C9382E390E07ED0A5E68C918F5FA6
:100250008C9308F4D7CF37980895C498C29AA8E62B
:100260008C918F5F8C9381E0809365000091650095
:10027000053010F009F00FC0C198E5E0F0E054D06F
:10028000C19AE1E0F0E050D0C198A5E68C918F5F73
:100290008C9308F4EBCFC29800916800033009F00A
:1002A00001C001C003CFC19882E090E04CD0C19A58
:1002B00085E090E048D0C198B9988CE291E043D0B5
:1002C000B19B0DC0B99A809169008F7780936900C6
:1002D00080E08093620080E080936800E7CEE3CF07
:1002E000C1988CE291E02FD0C19A8CE291E02BD0A2
:1002F000E3E0F0E019D0B19B0FC0B99A809169009A
:100300008F778093690080E080936200AAE633D003
:1003100080E080936800CACEE3CFED91FC91EF5F5F
:10032000FF4FFC93EE93089588EE93E00CD0319745
:10033000D9F708953197F1F70895689462F8089510
:10034000E89462F80895EF93FF93EE27E82BE92BEA
:1003500031F0E0E6F9E03197F1F70197D1F7FF913D
:10036000EF910895369A3699FECF369A3699FECF98
:1003700084B195B1089582E001C084E099279D93EE
:100380008A95E9F70895E199FECFEEBB319608957D
:1003900091E001C092E07B3751F47FB7F894F3DF2E
:1003A0008D918DBBE29AE19A9A95C9F77FBF772725
:1003B000089591E001C092E0E6DFE09A8DB38D935D
:0603C0009A95D1F70895A3
:00000001FF
